:020000040800F2
:1000000000800020FD160008471700087519000839
:1000100000000000000000000000000000000000E0
:1000200000000000000000000000000003170008AE
:100030000000000000000000051700083D0C00084B
:1000400007170008091700080B1700080D1700080C
:100050000F170008111700081317000815170008DC
:1000600017170008191700081B1700081D170008AC
:100070001F1700082117000823170008251700087C
:1000800027170008291700082B1700082D1700084C
:100090002F1700083117000833170008351700081C
:1000A00037170008391700083B1700083D170008EC
:1000B0003F170008411700084317000845170008BC
:1000C0004543532E46573A30312E30302E303100D2
:1000D0000120C006014908607047C04608ED00E0F5
:1000E00010B51D4CA0688006400F411E032923D87F
:1000F0001A48C0467944097949008F442201171AE9
:10010000E16803220A40032A00D01548E168490645
:10011000490F491C01F036FCE1684904490E484387
:10012000E168490F491C01F02DFC0AE07D20000226
:1001300007E00120C00304E020688004410F084864
:10014000C84008490860A26892093C231340064A47
:10015000D258D040086010BD0010024000127A0052
:0C0160000024F400200000206C010008C6
:10016C000000000000000000000000000000000083
:10017C000000000000000000000000000000000073
:10018C000100000002000000030000000400000059
:10019C000600000007000000080000000900000035
:1001AC00D0B502AFFFB08DB06E4600F0FDFA012560
:1001BC002804F062E807B0603561FC480068F06123
:1001CC00FB48FC4900F012FFFB4800F0FBFB7F28CA
:1001DC000FD080B2F949884203D0F949884200D146
:1001EC00A3E2F2480068F169401AF3498842E7D962
:1001FC009BE2F448EF4900F0F9FE01F0A1FBF24854
:10020C0000F0E0FB0446401CF9D0A0B2EC49884257
:10021C00D6D0ED4800F0D6FB0028F0D4FF21B16217
:10022C008143E2B2022A16D1022914D1E748E149EE
:10023C0000F0DCFEE64880194570792101700171EF
:10024C00E44A1178C17051780F220A40827005215E
:10025C0000F08EFCD3E71046084324D1DE48D54984
:10026C0000F0C4FEDA48801979218173922242731E
:10027C00822202737322C2726322827243224272FE
:10028C00312202722122C271112282710223437126
:10029C0005710023C37082700B22427001700F2114
:1002AC0000F066FCABE7112A16D1112914D1CB480A
:1002BC00C04900F09BFE01F043FB0024C8480471C8
:1002CC000460052C17D0C04800F07CFB002896D4A5
:1002DC00C3490855641CF4E7012A2ED101292CD1FD
:1002EC00BB488019792101710022C27082701122E1
:1002FC0042700170ABE7BA4CE078A1786278237851
:10030C0053404B404340206802BA2260207983421C
:10031C003CD1B448A74900F069FE01F011FB002460
:10032C00022C55D0A84800F04DFB002800D566E7FC
:10033C00A74989190855641CF2E7432A2DD1432992
:10034C002BD1A9489B4900F051FE01F0F9FAF8486D
:10035C0000F038FB002800D551E702460930072190
:10036C0088436946716169460D1AAD46941CB561A6
:10037C003262002C5CD0EE4800F024FB002800D543
:10038C00C4E028706D1C641E326AF2E79748F1498C
:10039C0000F02CFE01F0DEFA31E7312A39D1312997
:1003AC0037D1ED48E94900F021FE01F0C9FA0024EB
:1003BC00EA4804710460052C00D1AEE0DC4800F082
:1003CC0001FB002800D51AE7E4490855641CF2E744
:1003DC00F44880194578B16A4D400078A84200D0A5
:1003EC0097E02C4608340720844301F0A9FA6846AC
:1003FC00B0626846041BA5466D1CEC2220462946BB
:10040C0001F051FB2046294600F0B2FBB06A85464C
:10041C0081E0CF48CF4900F0E9FD01F09BFACA48D2
:10042C000068F169401AC349884200D8E7E67CE1CC
:10043C00551CD5482946144600F0D8FDE4B2B069E5
:10044C00F560002D0BD001787162B062CF4800F0DE
:10045C00CDFDB06A716A4C40401C6D1EF1E7CC4872
:10046C0000F0C4FDB069F168405C84426ED1B248C2
:10047C004068002805D5B0480838B0490160B1493A
:10048C000160C448B14900F0B1FD00223569306A01
:10049C00B16982425EDC8C5C062C35D3B262A64814
:1004AC000068F16A084204D0B448A84900F09EFDE7
:1004BC00F5E7A14A106810603F20C00051688143E5
:1004CC005160E00051680143516050680221716233
:1004DC00084350605068F16A0843506096480068C1
:1004EC00F16A08429949224603D0AB4800F07EFDE0
:1004FC00F4E7AA4800F07AFD8F494868726A904385
:10050C004860306AB169B26A521CC2E770698546AC
:10051C0001E001F01FFA356971E6904A10785178C4
:10052C00414090784840D17841401079814200D0C8
:10053C0030E701F005FA7E4800F044FA002800D5B7
:10054C005DE6411C8A0713D0854820E701F002FACA
:10055C0035690AE092487D4900F048FD764A5068BA
:10056C00B1680843506001F0EBF97069854646E6C6
:10057C007062B16229028B488019FF22316201F04E
:10058C0092FA0024B06AA04209D0694800F01AFA25
:10059C00002804D4834989190855641CF2E768487B
:1005AC000068C00724D0142023E0C046D8000020E7
:1005BC00642000089820000810270000FFFF0000AE
:1005CC00FEFF00001C1B0008881300002F1B0008F6
:1005DC003001000000580140A0200008B4200008A1
:1005EC00CC000020921D0008CE1D0008B01D000894
:1005FC00042053490D50706A844200DCFFE5044628
:10060C004B4800F0DFF9002800D5F8E50021224620
:10061C00A14205DC634B9B195B5C5A40491CF7E714
:10062C00D1B2814200D0B5E64C49086802BA0A60E2
:10063C004C4882421CD310194B49884218D8F01DE3
:10064C002930316A01F02EFA49484049B26A00F06B
:10065C00CDFC0024706A844210DC524880190019C9
:10066C00F11D29310A19434900F0EAFA1034F1E777
:10067C003E483849B36A00F0B9FCBEE52E484068E4
:10068C00002805D52C4808382C4901602D490160FB
:10069C0039482E49B46A224600F0A8FCE0103062BA
:1006AC000024306A844237DA23480068F16A084231
:1006BC0004D03248254900F099FCF5E71E4908683A
:1006CC0008600B46B462E400F01D2930011949683A
:1006DC0071620159214A126818465B682B434360CA
:1006EC0011511019BFF36F8F716A41601248006885
:1006FC00F16A084204D02248144900F077FCF5E76F
:10070C000D4800681548006802191E480F4900F092
:10071C006DFCB46A641CC4E7074A5068A843506077
:10072C005068B1680843506067E500F0ADF944E5E6
:10073C008813000010270000102002402301674599
:10074C0014040050AB89EFCDD8000020982000088D
:10075C00D61B0008D02000085F1F0008CC0000202A
:10076C00DC20000800300008FFEF01085E1E0008C6
:10077C001E1E000854200008381E0008701B0008BC
:10078C00042100089B1B0008461B0008D820000809
:10079C00E41D0008591B0008361F0008E61D000860
:0807AC00041E000830010000EA
:1007B400F0B585B0714800687D21C90001F0E0F80A
:1007C400401E010E0DD16E496E4A50606E4803689A
:1007D4000B4003218907591801600020906007200D
:1007E40010606A4800F006FC69486A496A4A00F0E9
:1007F40001FC0125AC02694E3068400507D430681D
:10080400204207D16F48704900F0F4FBF7E76448D1
:1008140000F0F0FB0394706B032210437063614E8D
:1008240030689043306030680C2102918843306016
:1008340030682843306030680421014331602B0460
:1008440005273C0758488169C9B2AA29049303D0F3
:100854008169C9B2CC292ED1216989042BD5C168FB
:10086400002903D551490160514901600192C168D1
:10087400490003D54F4941604F4941608169FF22D6
:10088400914381618169EC220A4382618168194242
:10089400FCD16904C2680A43C26081681942FCD170
:1008A400E906C2680A43C2600020C143642000F024
:1008B400A1F9049B019ACF2080042168814321601F
:1008C4004520C0042168014321601005E16881438B
:1008D400E1602805E1680143E1600F200102626ADA
:1008E4008A4362622902626A0A436262616AF0228E
:1008F40091436162616A10220A4362620004616A80
:1009040081436162606A18436062A903234A106CE0
:100914000843106429480268AA4302602A0703684E
:10092400934303602A03036813430360EA030368E1
:10093400934303600268039C224302600268029BA3
:100944001A43026002681E4B1343036082680A4321
:100954008260BF3CC460016829430160002F0BD052
:10096400B5619624204600F037F90498B06120461A
:1009740000F032F97F1EF1E705B0F0BD2000002041
:10098400FFFFFF0010E000E020ED00E0C11F0008C1
:100994005C21000898200008C000000800100240F4
:1009A400101C000800040050082002402301674581
:1009B400AB89EFCD3B2A19087F6E5D4C00380140AE
:0C09C4000000FF037421000894210008CB
:1009D000F0B581B026490B680A68264C2C4D266874
:1009E000B60611D40E68B61A86420DD20E68F61AF3
:1009F0004B2EF4D30B682E68F60701D0142600E0C6
:100A0000042601277751EAE70968891A81420FD243
:100A1000194D206800070FD42068400712D42068C1
:100A2000800715D42068C00718D1A068C5B21BE0A4
:100A30000020C043451E17E01048114900F0DCFAC1
:100A4000082010E00F480E4900F0D6FA04200AE012
:100A50000D480B4900F0D0FA022004E00B48084989
:100A600000F0CAFA0120606028B201B0F0BDC046B3
:100A7000D80000201C380140FFFF0000C41E000801
:100A8000D0200008E21E000840210008A41F000832
:040A900014040050FA
:100A9400F0B581B001200303274A1168009319437C
:100AA4001160264EB1680143B1602548254900F024
:100AB400A1FA0024244F2548844222490AD2E51988
:100AC4002B482A4600F096FAE05900BA30602948CB
:100AD4002C18F0E71E4800F08DFA1E4800683168B3
:100AE40081421FD11F48174900F084FA7D208000FD
:100AF40000F072F810490868009A904308601A4898
:100B0400002484604460046072B618480760386842
:100B140080F3088862B678688047E1437D2000F05E
:100B240069F8FAE70C480D4900F064FAFA200C4918
:100B340000F060F801B0F0BD38100240003002400F
:100B4400F11B00089820000800300008FCBF0100D9
:100B5400911F0008FCEF0108A01E0008D020000827
:100B6400881300002C21000810E000E008ED00E0EC
:080B74007C1F000804D0FFF70C
:100B7C00F0B581B00C4605460F481049224600F0EE
:100B8C0035FA00260E4FA6420CDA38680006FCD562
:100B9C00A85DF860282E03D8A95D0C4800F026FA51
:100BAC00761CF0E7282C01DC074800E0054800F033
:100BBC001DFA01B0F0BDC046AE1E0008982000081A
:100BCC001C3801409F1F0008E41D00089A1F0008F4
:100BDC0081B005490A6800920A68009BD21A8242C9
:0C0BEC00FAD301B07047C046D8000020CA
:100BF800F0B581B000910546012630040B4F3860EE
:100C08000B4804680A480068001B009988420AD209
:100C1800022038602846FFF7DDFF70043860284658
:100C2800FFF7D8FFEEE701B0F0BDC046180400504A
:040C3800D8000020C0
:100C3C0002480168491C01607047C046D80000207A
:100C4C00F0B591B00023102B03D0C45CD4545B1CC2
:100C5C00F9E7A3480160A34802600022A248102AC9
:100C6C000BD08B5C835483188C1865785D70A578D9
:100C7C009D70E478DC70121DF1E704219A4C2C294C
:100C8C0048D08D000C22102A06D0A35C10AEB618EA
:100C9C000C3E3370521CF6E710AEF778B3787278CE
:100CAC003678880703D00F970E93134612E08F48BF
:100CBC000D910146865D10A80F96C670CE5D0E96FE
:100CCC008670CB5C43708A5C0D998E08884FBE5D34
:100CDC0056400670844F7A191046103800787040D0
:100CEC0078550120284316460F3E36785E403E5418
:100CFC000220284313460E3B1B780E9E73403B5438
:100D0C00032028430D3A12780F9B5A403A54241D65
:100D1C00491CB4E70A2000F0EFF80920754C00904C
:100D2C0070480068417B427A427342794378437140
:100D3C00427241708178827A827081728179827B71
:100D4C0082718173C178C279C270C27AC271C27B5E
:100D5C00C173C272002104290AD00022102A04D0C7
:100D6C00835CE35C8354121DF8E7401C491CF2E7DA
:100D7C000099080600D1AEE0C8B200F0BDF85948A1
:100D8C00006807900020102800D1A1E007990A56AE
:100D9C000F46D109144604921B2211400B460F90AA
:100DAC006000434059001E4605934BB2DB091340CB
:100DBC0040B2C009104048404100054606905940D9
:100DCC000E910F98391801200F560B460220095628
:100DDC001C4603930846784070400323E3560C935B
:100DEC005840FB0913407C000D9463400A93584013
:100DFC006840CB0913404D006B400B935C00019491
:100E0C006DB2EE0916406640704002960E9B58403B
:100E1C000A9B5C0065B2EB0913400D9D6DB2ED09A8
:100E2C001540654009956C005C4008946040019B3E
:100E3C005BB2DB09134074005C400D9460400C9B6A
:100E4C00DC0914405B005C4065006EB2F60916408C
:100E5C005BB2DB0913406B405A00724050400F9D4F
:100E6C00079E70550846049D68400C9E70400A9E73
:100E7C0070400B9E7040099E70400E9E7040584012
:100E8C00089E70400D9E70405040039E70700F98ED
:100E9C006F406740174C0E9D6F407940059D69402F
:100EAC00099D69405940089D69400D9B594051402E
:100EBC00F1700C994F400B994F4006994F40029995
:100ECC004F406F400D994F405740B770001D5AE787
:100EDC000098401E23E7002000F00EF811B0F0BD82
:100EEC00EC000020D4000020F00400209C2100081D
:080EFC001F1C00089C220008E5
:100F040030B500010A4908180A4909680022042A70
:100F14000CD00023042B05D0C45CCD5C6540CD54BB
:100F24005B1CF7E7091D001D521CF0E730BDC046ED
:080F3400F0040020D4000020AD
:100F3C0003490868002801D1024808607047C04680
:080F4C00E80000200000002075
:100F54007F2805D8034A125C0348405C1040704760
:0C0F6400002070479C2300082720000894
:100F70007F2805D8034A125C0348405C1040704744
:0C0F8000002070479C2300082720000878
:100F8C00F0B503AF91B06E46F51D1935B3617261C2
:100F9C007160F06000F0A2FDB060C21D07218A43B1
:100FAC00694631616946881A30608546F41D1534EE
:100FBC002046716800F073FC0A48F0630A48286008
:100FCC00F0682862B06868613068E8602046716932
:100FDC00B26900F01FF831698D46FC1F053CA5462F
:0C0FEC00F0BDC046D91A0008FFFFFF7FCF
:100FF80083B010B581B0044603A80EC00548006848
:1010080003AA0092214600F055FC01B010BC02BCB6
:0810180003B00847140000209A
:10102000F0B599B00B920D46044600200490206064
:1010300013A8401E1290012001020A91410208915A
:1010400041030191810302910390C00306900C9427
:101050002978252907D0002900D14FE26D1C2046B0
:1010600000F0B9FBF4E7ED1C049F069C089EA81E47
:1010700000780246203A102A0FD880217A4412794B
:1010800052009744081919161919190F191927111F
:1010900019131919150040210BE05E280CD101200D
:1010A000010306E0214604E0202102E0102100E0D7
:1010B00031460F436D1CDAE76D1E002601463039BC
:1010C000C9B2092912D80A2171434618303E28783E
:1010D0006D1CF3E70B9901C90B91002801D5102174
:1010E0000F43C1174840461A681E00782E280CD1BD
:1010F00028782A2833D16878AD1C0B9A02CA0B9243
:10110000002903D40A9A174300E00021F21703468E
:10111000683BDC01DBB25B08E318DBB2092B39D892
:101120009B0002A4E3580C9C9F46C0465511000842
:101130007B11000885110008A5110008A511000801
:10114000A51100087F110008A5110008A5110008CD
:101150007F110008287868281ED1082016E06D1C31
:1011600000210246303AD2B2092AC9D80A224A439B
:101170008118303928786D1CF3E70220074328785E
:101180006D1C0FE028786C2809D10220074368788D
:10119000AD1C07E00C9C05E06D1C042301E06D1CF8
:1011A000039B1F4396430246633A152A17D8C0464D
:1011B0007A441279520097441A0B0A0A0A0A0B0A57
:1011C0000A0A0A2936440A0A530A650A0A743FE7DA
:1011D0000796029C2743002209923A4673E025288D
:1011E0005BD058285BD0002800D031E795E130462D
:1011F0000B9E3478421E0C983946119200F04AFB3F
:101200000C982146044600F0E6FA6CE138072168A4
:101210000B9A00D54CE1B8071068016000D449E191
:101220000021416046E107960A9A17423A4601D0EA
:10123000BE4B1A403B06DB1730241C400994029C2D
:1012400041E0079638060A990F43C0172321014051
:1012500009910B9810C80B90002308200590D9E045
:1012600007960B9800680028B34E00D006463C460F
:10127000AE4804400A980742304600D01DE100F015
:101280009CFA1CE10A9A1742079601D0A74A174018
:101290003A46029C0023099315E02521DFE6019AD6
:1012A0001743A14B782800D12033029C3A06D2176D
:1012B00009920A9A1742079601D09C4A17403A466B
:1012C000099F1F4009970B9E02231340224204D11D
:1012D000002B07D1331D00240AE0002B11D108CECA
:1012E000DF1713E0F61D07239E4374683346083367
:1012F0003768560711D40F97160711D5FCB20F9413
:101300000DE0F61D07239E4388CE0036540709D40E
:1013100014070AD40F933C460BE0BFB20F9700248A
:101320001E4619E01CB21B0401E05CB21B060F94C0
:10133000DC17002C05D493060CD453060CD52023BF
:1013400009E000230F9F7F420F97A3412D270997A4
:101350001C4601E02B2309930B960A9B1A4201D0ED
:10136000724B1A40174623460A9A1742039A0F9C5B
:1013700000D00A46059201466F390026092916D881
:101380007944097949008F440445595959591859E4
:1013900059452046184351D007202040303013A92A
:1013A0008855E00859074418DB08761CF1E75828EF
:1013B00030D0642801D0692840D1394606980140D0
:1013C0000D912046184339D00D98002807D00320EE
:1013D0003040032803D113A82C218155761C0A2004
:1013E00011900020109020461946119A109B00F091
:1013F000E5FA0E900F940C46119A109B00F0C3F979
:1014000023460F99081A3021014313A88155761CF1
:101410000E9CD6E701980742454800D04548002673
:10142000214619430AD00F212140415C13AA91554E
:1014300021091A078C181B09761CF1E7099C611E0B
:10144000204688410799891BFF2C00D9491E081A9C
:1014500005998B1BD9178B43C21A08980742109322
:1014600006D10C98394600F015FA0020119000E0E2
:101470001192210A02D00C9800F0ADF9002C2146FF
:101480000C9C02D0204600F0A6F920463946119A5D
:1014900000F000FA30212046109A00F0EEF9012EFB
:1014A00023DB1298815D204600F095F9761EF6E761
:1014B00010680170121D0B92CAE500F003FB07468D
:1014C0000798C21B0C982146119200F0E3F9002FF7
:1014D00006D031780C9800F07EF9761C7F1EF6E776
:1014E00027460C9C0B9E361D0B96F80600D4AFE5E4
:1014F00020212046119A00F0C0F9A9E5E0680028F3
:1015000005D006CC083C914201D2049A42542046B0
:1015100000F0A6F9206819B0F0BD204600F0A0F94F
:101520000020C043F7E7C04658300000FFFDFFFF32
:0C1530002C2400081C2400088B1D00085F
:10153C00084B02001B680020934209D0064B1B6825
:10154C00934205D0054B1868801A431E98414042BF
:10155C007047C04618000020140000201C0000201A
:10156C000322104B30B510491A615A610F4A996128
:10157C00DA618022D2001A6200229A625A62DA621E
:10158C0019660B490B4C5966102199661A67DA6675
:10159C005A670F321500105DA91A5854013AFAD245
:1015AC0030BDC0462400002034200008F00000208C
:0815BC00A00500203D200008FD
:1015C400F8B516001822451C55434243164B0F002C
:1015D400ED189B18DC6A012C10D0022C1BD0002CB7
:1015E4001FD1280000F07AF9864205D8320039006C
:1015F400280000F079FA34002000F8BD280000F03B
:101604006DF93400864200D9040022003900280014
:1016140000F06AFAF0E73200280000F068F90400EC
:0C162400EAE70024E8E7C04624000020AC
:10163000F8B50B4B04001B780E001700002B01D1EE
:10164000FFF794FFEFF31085012181F310883A0032
:1016500031002000FFF7B6FF85F31088F8BDC046C3
:041660002400002042
:0C166400F81E0008901600087016000820
:10167000550F0008811A00088D1A0008710F000824
:10168000991A0008A51A0008711A0008451A0008DE
:10169000FA1E000814200008142000081420000876
:1016A000142000081420000814200008142000084A
:1016B0001420000814200008FFFFFFFFFFFFFFFFBA
:1016C000FFFFFFFFFFFF0000FC1E0008C61F000811
:1016D0001E1D0008E31F0008751D000815200008E6
:0816E0001E2000087C1D00081B
:1016E800034C206804348047FBE7FEF75BFDFEE708
:0416F8003C24000886
:0616FC00FEF7E8FCF2E736
:02170200FEE700
:02170400FEE7FE
:02170600FEE7FC
:02170800FEE7FA
:02170A00FEE7F8
:02170C00FEE7F6
:02170E00FEE7F4
:02171000FEE7F2
:02171200FEE7F0
:02171400FEE7EE
:02171600FEE7EC
:02171800FEE7EA
:02171A00FEE7E8
:02171C00FEE7E6
:02171E00FEE7E4
:02172000FEE7E2
:02172200FEE7E0
:02172400FEE7DE
:02172600FEE7DC
:02172800FEE7DA
:02172A00FEE7D8
:02172C00FEE7D6
:02172E00FEE7D4
:02173000FEE7D2
:02173200FEE7D0
:02173400FEE7CE
:02173600FEE7CC
:02173800FEE7CA
:02173A00FEE7C8
:02173C00FEE7C6
:02173E00FEE7C4
:02174000FEE7C2
:02174200FEE7C0
:02174400FEE7BE
:0E17460080B50020C143FA20FFF753FA80BDA2
:10175400F0B581B00EB470BC07461846FFF7ECFE36
:101764000146002000290AD46543A54207D3304628
:1017740039462A4600F0ADF8214600F001F901B0DF
:02178400F0BDB6
:1017860030B5514343435C18010C130C0D005D4307
:10179600641992B2514380B242430D0C09045218A7
:0E17A60065415843010C00048018694130BDB4
:0617B40000200021704737
:0E17BA00411C02780130002AFBD1401A704712
:0E17C800002A03D0013A8B5C8354FBD170479A
:1017D60030B581B0044668460170206900280FD0F4
:1017E6000CCC083C9A4233D26269531C6361815423
:1017F600A069616981422BD1204600F02EF827E0CE
:10180600E068002809D00CCC083C9A4220D2551C2E
:101816009D4200D1002181541AE0A068002808D01A
:101826000CCC083C9A4213D2551C9D420DD0C9B22D
:101836000CE0236A002B0BD003CC083C884207D26D
:10184600694601222046984702E000219200815015
:0A1856002068401C206001B030BD86
:1018600010B54269002A07D00446036A002B01D054
:0A187000216998470020606110BD57
:10187A0070B514460D460646012C05DB304629464E
:0A188A00FFF7A4FF641EF7E770BD2E
:1018940080B5CB0606D4890501D5302100E020218E
:0618A400FFF7E9FF80BD23
:1018AA00B0B50C4605460021242200F000F9EC618F
:0218BA00B0BDBF
:1018BC0070B514460D460646FFF73AFB0146304616
:0A18CC002A462346FFF75CFB70BDBF
:0A18D60010B50068FFF7A9FE10BD71
:1018E0000369C268934201D881685B18013B981A6A
:0218F00070473F
:1018F2000023F7B506001700C5680191009333690C
:10190200B4689D421FD2013B5B1B641BBC4200D9E1
:101912003C009C4200D91C007068220040190199C9
:10192200FFF751FF009B2D191B190093019B3F1BD1
:101932001B190193B368AB4200D10025F560002F5B
:0A194200DDD10098FEBD1B19DDE7A2
:10194C0000B581B06846792101700121FFF710F9CB
:04195C0001B000BD19
:1019600000B581B068461F2101700121FFF706F91B
:0419700001B000BD05
:1019740080B57D2080000021C943FFF73BF980BD7D
:101984000A0015D00300400800E052008242FCD94E
:10199400002000E052089B1A06D340418A42F9D144
:1019A400704752089B18F8D200188A42F9D1704740
:0819B40010B5FFF7FDFE10BDA8
:1019BC0070B400240125ED07002B07D1002905D0B8
:1019CC00834203D2130000222C0000250026A41908
:1019DC00994200D1904212D992185B4103D2EE0782
:1019EC006D086408F3E7DE075B08520892190126BC
:1019FC00F6079B1903E0DE075B0852089219801A60
:101A0C00994103D364416D41F5D30FE024196D4125
:101A1C000AD2DE075B085208921980185941F5D397
:101A2C0064416D41E7D301E08018594102000B007D
:081A3C002000290070BC704776
:101A440010B5002A0DD00446097848B200280AD4FB
:101A5400002C00D02160002119605960411E88418A
:0C1A640010BD002010BD0120C04310BDCB
:101A7000024601207F2901D9C04370471170704789
:0C1A8000014661391A2900D22038704755
:0C1A8C00014641391A2900D22030704771
:0C1A9800014661391A2900D2203870473D
:0C1AA400014641391A2900D22030704759
:101AB00000220B0011001A00002A02D0013A8154C2
:041AC000FCD170479E
:101AC40002460020135C002B03D0814201D0401C4D
:041AD400F8E7704778
:101AD80010B50C46436A01212046FFF737FE10BDBA
:041AE80040207047E3
:101AEC00F7B58368C468050040681F1B00190E0019
:101AFC000193A418974207D83A00FFF75FFE019BA9
:101B0C006868E41A2200F119FFF758FEEC60F7BD83
:101B1C002573424C20696E697469616C697A6564DD
:031B2C002E0A007E
:101B2F002573476F74204745545F494420636F6D99
:071B3F006D616E642E0A00C7
:101B46000945726173696E67202564207061676557
:031B5600733A00DF
:101B5900090925735374617274696E67206572612E
:071B690073696E672E0A008C
:101B700009257357616974696E6720666F722072F8
:101B8000656C656173696E67206F6620464C4153D2
:0B1B900048206D656D6F72792E0A0011
:101B9B0009257350726F6772616D6D696E67206F87
:101BAB0066203820627974657320617420616464E7
:101BBB0072657373203078253038582070657266E3
:0B1BCB006F726D6564206F6B2E0A00C6
:101BD6002573556E6B6E6F776E20636F6D6D616EDC
:0B1BE6006420307825303258210A00BE
:101BF10025735374617274696E672063616C6375D8
:0F1C01006C6174696E67204657204352430A0096
:0F1C10004853492069732072656164792E0A0078
:101C1F008D01020408102040801B366CD8AB4D9A02
:101C2F002F5EBC63C697356AD4B37DFAEFC5913981
:101C3F0072E4D3BD61C29F254A943366CC831D3AAB
:101C4F0074E8CB8D01020408102040801B366CD83D
:101C5F00AB4D9A2F5EBC63C697356AD4B37DFAEF4E
:101C6F00C5913972E4D3BD61C29F254A943366CCC6
:101C7F00831D3A74E8CB8D01020408102040801BAD
:101C8F00366CD8AB4D9A2F5EBC63C697356AD4B30A
:101C9F007DFAEFC5913972E4D3BD61C29F254A9495
:101CAF003366CC831D3A74E8CB8D010204081020F3
:101CBF0040801B366CD8AB4D9A2F5EBC63C69735F0
:101CCF006AD4B37DFAEFC5913972E4D3BD61C29F77
:101CDF00254A943366CC831D3A74E8CB8D010204F8
:101CEF0008102040801B366CD8AB4D9A2F5EBC631A
:101CFF00C697356AD4B37DFAEFC5913972E4D3BD77
:0F1D0F0061C29F254A943366CC831D3A74E8CB9A
:101D1E004A616E756172790046656272756172799B
:101D2E00004D6172636800417072696C004D61799B
:101D3E00004A756E65004A756C790041756775735A
:101D4E00740053657074656D626572004F63746FD5
:101D5E00626572004E6F76656D62657200446563F2
:071D6E00656D626572000063
:071D7500414D00504D00003C
:0F1D7C002561202562202565202554202559004A
:071D8B00286E756C6C290045
:101D92000925734164647265737320307825303885
:0E1DA20058207265717565737465642E0A00B1
:101DB0000A2573204D656D6F7279206164647265C8
:0E1DC000737320435243206572726F722100CC
:101DCE002573476F7420455241534520636F6D6DE7
:061DDE00616E642E0A0094
:021DE4000A00F3
:101DE60009092573506167652025642068617320A1
:0E1DF6006265656E206572617365642E0A0079
:101E04000909257345726173696E672069732066D9
:0A1E1400696E69736865642E0A00A8
:101E1E0009257344656372797074696E6720256451
:0A1E2E002062797465732E2E2E00D9
:101E38000925735374617274696E672070726F67D5
:101E480072616D6D696E67206F6620256420627906
:061E58007465732E0A0000
:101E5E002573466F7262696464656E206164647294
:101E6E00657373206F662030782530385820666F82
:101E7E00722077726974696E67206F662025642000
:101E8E00627974657320726571756573746564210A
:021E9E000A0038
:0E1EA0002573435243206572726F72210A004F
:101EAE0009257353656E64696E6720256420627917
:061EBE007465733A200078
:101EC40025734F76657272756E206572726F72201B
:0E1ED4006973206465746563746564210A0097
:101EE20025734E6F69736520697320646574656339
:061EF200746564210A0082
:021EF8004300A5
:021EFA002E00B8
:101EFC0053756E646179004D6F6E64617900547531
:101F0C006573646179005765646E6573646179000B
:101F1C005468757273646179004672696461790002
:0A1F2C00536174757264617900005E
:101F36000909257357616974696E6720666F722097
:101F46007061676520256420746F20626520657264
:091F5600617365642E2E2E0A0051
:101F5F002573476F74205752495445204D454D4FB7
:0D1F6F00525920636F6D6D616E642E0A0083
:101F7C000D257309416464726573733A20307825BA
:051F8C00303858200070
:091F91002573446F6E65210A00FE
:051F9A00253032580063
:051F9F002E2E2E0A00A9
:101FA4002573506172697479206572726F72206949
:0D1FB40073206465746563746564210A0020
:051FC1001B5B324A0029
:101FC60053756E004D6F6E0054756500576564005D
:0D1FD6005468750046726900536174000084
:101FE3004A616E00466562004D6172004170720085
:101FF3004D6179004A756E004A756C004175670042
:10200300536570004F6374004E6F76004465630040
:0120130000CC
:0120140000CB
:09201500256D2F25642F257900AB
:09201E0025483A254D3A255300EE
:0D2027000007032004170201085710408035
:092034005465726D696E616C0067
:10203D0000000000000054545220524547474553BC
:01204D000092
:04205000E1000008A3
:10205400046062063E0B5C4E040620504F34414B34
:1020640025730A57616974696E672031307320667D
:102074006F7220636F6D6D756E69636174696F6EE5
:1020840020696E697469616C697A6174696F6E2E16
:042094002E2E0A00E2
:082098001B5B313B33326D008C
:1020A0002573476F742047455420636F6D6D616ED3
:0420B000642E0A0090
:1020B4002573476F7420524541445F4D454D4F523F
:0C20C4005920636F6D6D616E642E0A0080
:0820D0001B5B313B33316D0055
:0420D800202564005B
:1020DC000925734279746573206E756D6265722083
:1020EC006D757374206279206D756C7469706C6594
:0820FC00206F662034210A0068
:1021040009257357616974696E6720666F7220745C
:10211400686520656E64206F662070726F677261F7
:082124006D6D696E672E0A0063
:10212C002573094352437320617265206571756193
:04213C006C2E0A00FB
:1021400025734672616D65206572726F72206973C6
:0C215000206465746563746564210A00F6
:10215C00257350726F6772616D2073746172746550
:08216C006420282573290A00F4
:10217400257357616974696E6720666F72204853CE
:102184004920746F206265207265616479210A00B8
:082194001B5B323B33336D008D
:10219C00637C777BF26B6FC53001672BFED7AB7618
:1021AC00CA82C97DFA5947F0ADD4A2AF9CA472C0C3
:1021BC00B7FD9326363FF7CC34A5E5F171D8311530
:1021CC0004C723C31896059A071280E2EB27B27551
:1021DC0009832C1A1B6E5AA0523BD6B329E32F84C9
:1021EC0053D100ED20FCB15B6ACBBE394A4C58CFC1
:1021FC00D0EFAAFB434D338545F9027F503C9FA895
:10220C0051A3408F929D38F5BCB6DA2110FFF3D262
:10221C00CD0C13EC5F974417C4A77E3D645D197316
:10222C0060814FDC222A908846EEB814DE5E0BDB10
:10223C00E0323A0A4906245CC2D3AC629195E47947
:10224C00E7C8376D8DD54EA96C56F4EA657AAE08A1
:10225C00BA78252E1CA6B4C6E8DD741F4BBD8B8A3C
:10226C00703EB5664803F60E613557B986C11D9EA2
:10227C00E1F8981169D98E949B1E87E9CE5528DF19
:10228C008CA1890DBFE6426841992D0FB054BB1645
:10229C0052096AD53036A538BF40A39E81F3D7FBCF
:1022AC007CE339829B2FFF87348E4344C4DEE9CB19
:1022BC00547B9432A6C2233DEE4C950B42FAC34E8E
:1022CC00082EA16628D924B2765BA2496D8BD12544
:1022DC0072F8F66486689816D4A45CCC5D65B692E8
:1022EC006C704850FDEDB9DA5E154657A78D9D848C
:1022FC0090D8AB008CBCD30AF7E45805B8B34506AC
:10230C00D02C1E8FCA3F0F02C1AFBD0301138A6BC5
:10231C003A9111414F67DCEA97F2CFCEF0B4E673F5
:10232C0096AC7422E7AD3585E2F937E81C75DF6EA3
:10233C0047F11A711D29C5896FB7620EAA18BE1B09
:10234C00FC563E4BC6D279209ADBC0FE78CD5AF4AF
:10235C001FDDA8338807C731B11210592780EC5FF5
:10236C0060517FA919B54A0D2DE57A9F93C99CEF51
:10237C00A0E03B4DAE2AF5B0C8EBBB3C8353996152
:10238C00172B047EBA77D626E169146355210C7D90
:10239C0020202020202020202068282828282020C9
:1023AC002020202020202020202020202020202021
:1023BC0048101010101010101010101010101010D9
:1023CC008484848484848484848410101010101079
:1023DC0010818181818181010101010101010101D2
:1023EC000101010101010101010101101010101086
:1023FC0010828282828282020202020202020202A3
:10240C00020202020202020202020210101010204A
:10241C00303132333435363738394142434445460E
:10242C00303132333435363738396162636465663E
:10243C008D24000824000020AD0000008D2400082D
:10244C00D4000020DC0400009F24000800000020C1
:0C245C006824000824000000F3160008AB
:10246800641600086416000864160008641600085C
:1024780064160008DC000020E0000020E4000020D2
:042488000024F40038
:10248C00206861680834002200E042540139FCD510
:02249C00704787
:10249E0020686168A2680C3401E08B5C8354013AB9
:0424AE00FBD57047A3
:04000005080016FDDC
:00000001FF
